:0400000040EF15F0C8
:1000080000C017F00CC016F00DC015F0E1CF18F0C5
:10001800E2CF19F09EAA50D09DAA4ED0AFCFC2F021
:10002800ACA202D0AC98AC88ACA404D0AFCFC2F0DC
:100038003F0EAE6E010E0001C95D02E17F0EC85D84
:1000480004E2C2510D0A01E025D0C8C0CCF0C9C0F5
:10005800CDF0C26B010EC36F000EC46FCD0EC82564
:10006800E16E030EC921E26EE1CFE1FFE2CFE2FFCC
:10007800E66AEA0E0C6EC30E0D6E0D2EFED70C2E20
:10008800FCD7AFCFC2F0C2510A0AD8B4C26BC86B52
:10009800C96B12D0CD0EC825E16E030EC921E26EE0
:1000A800E1CFE1FFE2CFE2FFC2C0E6FFC8C0CCF07B
:1000B800C9C0CDF0C84BC92BA4AA5ED0A3AA5CD0F6
:1000C8009CA202D09C989C889CA402D0AACF7FF5C1
:1000D800AACF7FF505017F510A0A18E1010E000138
:1000E800B26F000EB36F490ECA25E16E020ECB2126
:1000F800E26EE1CFE1FFE2CFE2FF7FC5E6FFCAC0D3
:10010800B4F0CBC0B5F005017F6B13D0490E0001E8
:10011800CA25E16E020ECB21E26EE1CFE1FFE2CF0C
:10012800E2FF7FC5E6FFCAC0B4F0CBC0B5F0CA4B4A
:10013800CB2B0001010ECB5D02E1800ECA5D1CE3F2
:10014800020EB26F000EB36FA39A010ECA5F000EC3
:10015800CB5B490ECA25E16E020ECB21E26EE1CFE0
:10016800E1FFE2CFE2FFE66ACAC0B4F0CBC0B5F067
:10017800CA6BCB6B05017F6BF2AA1AD0F2A418D018
:1001880001012C4B2D2B000E006E2D51005C02E15D
:100198002C51060808E2010E876F000E886FF29A4C
:1001A8002C6B2D6BD59E480ED76EE50ED66EF2944D
:1001B8009DA01BD09EA019D00101934B942B000E3B
:1001C800006E9451005C02E19351640804E2240E2D
:1001D800AE6E936B946B010E956F000E966FCD907B
:1001E8006D0ECF6E840ECE6E9E9017C000F016C0B6
:1001F8000CF015C00DF018C0E1FF19C0E2FF1100A6
:100208000B820BAE0EEF01F003680268016800680C
:080218000A360232FF0E12004B
:0E022000026A016A006A086A036A000E120090
:10022E000B840BAE22EF01F0010E036E026A016A1F
:0A023E00006A0A360232FF0E1200B9
:080248000AAE029E000E120036
:100250000CB06AEF01F00CA210EF02F00E6A000E73
:10026000026481EF01F0F00E0214D8A44CEF01F00B
:10027000023A01380F0B02260138F00B016E0038EC
:100280000F0B01260038F00B006E08380F0B00260C
:100290000838F00B086E0E84D89002BE65EF01F0AE
:1002A00008360036013602360E2A02BE65EF01F02E
:1002B00008360036013602360E2A02BE65EF01F01E
:1002C00008360036013602360E2A0E50036406EF59
:1002D00002F0035E0BBC08AE0BEF02F0D880800E7C
:1002E00008640030000E002201220222D8A00BEF89
:1002F00002F0023201320032034A10EF02F00BEF3B
:1003000002F001C002F000C001F008C000F0086A6D
:10031000000E0E860264B8EF01F0F00E0214D8A4AD
:10032000A0EF01F0023A01380F0B02260138F00B62
:10033000016E00380F0B01260038F00B006E0E84A2
:10034000D89002BE65EF01F00036013602360E2A63
:1003500002BE65EF01F00036013602360E2A02BEFB
:1003600065EF01F00036013602360E2A65EF01F026
:1003700001C002F000C001F0006A000E0E960E8867
:100380000264E5EF01F0F00E0214D8A4D0EF01F002
:10039000023A01380F0B02260138F00B016E0E8471
:1003A000D89002BE65EF01F0013602360E2A02BE79
:1003B00065EF01F0013602360E2A02BE65EF01F04C
:1003C000013602360E2A65EF01F001C002F0016A23
:1003D000000E0E86026415EF02F0F00E0214D8A48F
:1003E000F4EF01F0023A0E84D89002BE65EF01F0FE
:1003F00002360E2A02BE65EF01F002360E2A02BE58
:1004000065EF01F002360E2A65EF01F0010E0C6E69
:100410000EDF18EF02F0020E0C6E16DF18EF02F07E
:10042000040E0C6EF1DE18EF02F0080E0C6EF8DE12
:020430001200B8
:100432000B800BAE25EF02F0026A0AAEFF0E026ECF
:0C044200016E006E0A360232FF0E12003E
:10044E00086A096A100E0C6E01340836093604501B
:10045E00085E0550D8A0053C095ED8B007D0045000
:10046E0008260550D8B0053C0926D890003601362E
:06047E000C2EEAD712006B
:100484000C6A0E6A0250D8A45BEF02F001C002F0BD
:1004940000C001F0006A0E860250D8A45BEF02F09F
:1004A40001C002F0016A0E960E880250D8B46DEFB6
:1004B40002F00E50035ED8A4D8A072EF02F0D890D8
:1004C40002BE77EF02F0003601360236032E62EFE9
:1004D40002F072EF02F0010E0C6EA0DE7AEF02F071
:1004E400020E0C6EA2DE7AEF02F0040E0C6EAADE8F
:0204F4001200F4
:1004F600F4C500F00501F407005228E0F0C5E9FF55
:10050600F1C5EAFFEE50000A0CE0F0C5E9FFF1C5BF
:10051600EAFFF2C5D9FFF3C5DAFFEE50DE1801E1B6
:100526000FD0F0C5E9FFF1C5EAFFF2C5D9FFF3C563
:10053600DAFFDE50EE5C006E016A000E015A08D04A
:100546000501F04BF12BF24BF32BD2D7006A016A6F
:02055600120091
:10055800025006180E6E086A096A0B6A035007648F
:100568009FEF03F006500A6E068E028E03500B6E44
:100578000750036E000E0B64EFEF02F00B50075E9E
:10058800D8B490EF03F0070E07645EEF03F0075E40
:1005980000C008F001C000F002C001F0026A074E76
:1005A80090EF03F0076433EF03F0075E00C008F034
:1005B80001C000F0016A074E90EF03F0076411EFE5
:1005C80003F0075E00C008F0006A074E90EF03F0E2
:1005D8000764F8EF02F00AC002F005C001F004C099
:1005E80000F0086AB9EF04F0030E076403EF03F0A4
:1005F800075E08380F0B086E074E90EF03F0D8908F
:100608000832074E90EF03F0D8900832074E90EF6B
:1006180003F0D890083290EF03F0030E076422EF3E
:1006280003F0075E08380F0B086E0038F00B082639
:1006380000380F0B006E074E90EF03F0D890003291
:100648000832074E90EF03F0D89000320832074E78
:1006580090EF03F0D8900032083290EF03F0030EC9
:1006680007644AEF03F0075E08380F0B086E00387E
:10067800F00B082600380F0B006E0138F00B00262F
:1006880001380F0B016E074E90EF03F0D89001323E
:1006980000320832074E90EF03F0D8900132003252
:1006A8000832074E90EF03F0D8900132003208323A
:1006B80090EF03F0030E07647BEF03F0075E083842
:1006C8000F0B086E0038F00B082600380F0B006E71
:1006D8000138F00B002601380F0B016E0238F00BC1
:1006E800012602380F0B026E074E90EF03F0D890E8
:1006F8000232013200320832074E90EF03F0D890F0
:100708000232013200320832074E90EF03F0D890DF
:100718000232013200320832096A000E0EAE84EF4E
:1007280004F0081E001E011E021E082A00220122D3
:10073800022284EF04F00750D8A4A5EF03F0B9EF24
:1007480004F0096A02C00AF0028E068E0750035CA4
:10075800076ED8B477EF04F0070E076445EF04F08E
:10076800075E0450096E0550046E0650056E066A51
:10077800074E77EF04F0070E07641AEF04F0075EE0
:100788000450096E0550046E056A074E77EF04F0B1
:10079800070E0764F8EF03F0075E0450096E046A59
:1007A800074E77EF04F0070E0764DFEF03F00AC087
:1007B80002F0B9EF04F0030E0764EAEF03F0075EF6
:1007C80009380F0B096E074E77EF04F0D8900932FD
:1007D800074E77EF04F0D8900932074E77EF04F010
:1007E800D890093277EF04F0030E076409EF04F09C
:1007F800075E09380F0B096E0438F00B0926043818
:100808000F0B046E074E77EF04F0D89004320932CC
:10081800074E77EF04F0D89004320932074E77EF8D
:1008280004F0D8900432093277EF04F0030E07641D
:1008380031EF04F0075E09380F0B096E0438F00B2E
:10084800092604380F0B046E0538F00B042605380A
:100858000F0B056E074E77EF04F0D890053204327F
:100868000932074E77EF04F0D89005320432093286
:10087800074E77EF04F0D89005320432093277EF4B
:1008880004F0030E076462EF04F0075E09380F0BEB
:10089800096E0438F00B092604380F0B046E05386E
:1008A800F00B042605380F0B056E0638F00B0526ED
:1008B80006380F0B066E074E77EF04F0D890063215
:1008C800053204320932074E77EF04F0D890063229
:1008D800053204320932074E77EF04F0D890063219
:1008E800053204320932086A000E0EAE84EF04F0B5
:1008F800091E041E051E061E092A042205220622B8
:1009080009500826045000220550012206500222F0
:100918000EBE9BEF04F0D8A0AAEF04F00232013219
:1009280000320832033EAAEF04F0B4EF04F0D8B066
:10093800AFEF04F0000E081E001E011E021E082A5A
:100948000022012202220A7EAFEF04F0010E0C6E93
:100958007BDCBBEF04F0020E0C6E76DCBBEF04F020
:10096800040E0C6E4DDCBBEF04F0000E0C6E120092
:0E097800ADB202D00000FCD7F0C5AEFF1200F9
:10098600F0C5E9FFF1C5EAFFEE500501F21905E1F0
:10099600F0C500F0F1C501F010D0F0C500F0F1C5CA
:1009A60001F0F04BF12B00C0E9FF01C0EAFFEECFEA
:0C09B60000F00052E5E1006A016A120046
:0E09C200A8B202D00000FCD7F0C5A9FF1200B9
:0809D0000B6A0B86FF0E1200FA
:1009D800F0C502F0F1C503F002C000F003C001F059
:1009E800024A032A00C0E9FF01C0EAFFEE5201E013
:1009F800F3D70501F051025C006EF1510358016E06
:0A0A0800010E005E000E015A1200FC
:100A12000A6A0350D8A40A800750D8A40A820A504E
:100A2200D8B46CEF05F0030AD8B425EF05F00AB08C
:100A320020EF05F006AE6AEF05F068EF05F002AEB2
:100A420068EF05F06AEF05F00250800B0A6E029E15
:100A52000650800B069E0A18D8B436EF05F00A50ED
:100A6200D8B468EF05F06AEF05F00750035CD8B41C
:100A720040EF05F0D8A05CEF05F062EF05F00650FC
:100A8200025CD8B44AEF05F0D8A05CEF05F062EF43
:100A920005F00550015CD8B454EF05F0D8A05CEF26
:100AA20005F062EF05F00450005CD8B46CEF05F07D
:100AB200D8B062EF05F00A52D8B46AEF05F068EFD9
:100AC20005F00A52D8B468EF05F06AEF05F0D88055
:0E0AD2001200D8901200D880D88412001200B2
:100AE0000501ED6B050EED5D0AE2ED51EB25E16EC2
:100AF000000EEC21E26E200EE66EED2BF3D7ED51E9
:100B0000EB25E16E000EEC21E26EE66AED07ED5199
:100B1000EB25EE6F000EEC21EF6F0A0E046E000E57
:100B2000056EE9C500F0EAC501F091DC08C000F0EF
:100B300009C001F0300E0026EEC5E1FFEFC5E2FF6F
:100B400000C0E6FF0A0E046E000E056EE9C500F057
:100B5000EAC501F07CDC00C0E9F501C0EAF5000E51
:100B6000011802E1000E001801E102D0ED07CFD715
:020B7000120071
:100B72000B6A0350D8B4FFEF05F002500A6E028EE2
:100B82008E0E035E03AE03EF06F0036C080E035CE9
:100B9200D8A0DEEF05F0036E013602C001F0026A52
:100BA200080E035CD8A0DEEF05F0036E0136016A81
:100BB2000350D8A4D890E8EF05F00350D8B4E8EF7A
:100BC20005F0D89002320132032EE2EF05F00BBCA1
:100BD20001A0F5EF05F0D8A0F5EF05F0012AD8B491
:100BE200022A02BE12EF06F00AAE17EF06F0021E4C
:100BF200011E012AD8B4022A17EF06F0026A016A1E
:100C020017EF06F00B800BAE1BEF06F0026A0AAE7E
:100C12001BEF06F0FF0E026E016E0A3602321BEF68
:100C220006F0010E0C6E04DC1DEF06F0000E0C6ED9
:100C32001DEF06F0FF0E0C6E0150006E0250016EA9
:020C420012009E
:100C44000450000A12E10550000A0FE10650000AA0
:100C54000CE10750000A09E1FF0E006EFF0E016E61
:100C64007F0E026EFF0E036EA7D0086A096A075052
:100C7400D8B4CDEF06F00350D8B4D1EF06F002504B
:100C840006180A6E028E068E0E6A02C008F001C0B3
:100C94000CF000C00DF004500D5E0550D8A0053CCA
:100CA4000C5E0650D8A0063C085E086A0C6A0D6A01
:100CB400D8A064EF06F0D890023201320032083234
:100CC400010E0E6E0750035ED8A071EF06F07E0E83
:100CD4000E240326D8B0D6EF06F077EF06F07E0E8A
:100CE4000E240326D8A0DBEF06F0180E0B6E0D368B
:100CF4000C3608360036013602360E360450005ED5
:100D04000550D8A0053C015E0650D8A0063C025E02
:100D140006340E120EA092EF06F00D809DEF06F041
:100D2400045000260550D8B0053C01260650D8B022
:100D3400062802260D900B2E79EF06F0C3EF06F07D
:100D4400D8900036013602360E360450005E055047
:100D5400D8A0053C015E0650D8A0063C025E0634CD
:100D64000E10010B0D26D8B00C2AD8B4082AD8A42A
:100D7400C3EF06F008320C320D32032AD8B4D6EF92
:100D840006F00AAE089E0850026E0C50016E0D501B
:100D9400006EDEEF06F0010E19DEDEEF06F0020E45
:100DA40010EC01F0DEEF06F0040E04EC01F0DEEFCF
:0A0DB40006F0080E17EC01F0120023
:0E0DBE00570E0D6E0D2EFED700000000120025
:100DCC00086A096A000E076203646BEF07F00250B1
:100DDC0006180A6E075003267E0ED8A0FCEF06F00C
:100DEC00035ED8B070EF07F000EF07F0035ED8A0F9
:100DFC0075EF07F0028E068E02C00EF001C00BF0EC
:100E0C0000C00DF000500402F4CF0CF001500502AC
:100E1C00F4CF00F0F3CF08F00402F3500C26F4509A
:100E2C000822000E00220D500502F3500C26F4503F
:100E3C000822000E002202500402F3500826F4503F
:100E4C00002202500502016A000E0122F350002616
:100E5C00F45001220D500602F3500826F4500022E3
:100E6C00026A000E012202220B500602F3500026E9
:100E7C00F4500122000E02220E500602F3500126FD
:100E8C00F450022202BE53EF07F00836003601364A
:100E9C0002360306D8B475EF07F066EF07F0D8807A
:100EAC00800E08640030000E002201220222D8A01D
:100EBC0066EF07F0023201320032034A70EF07F09E
:100ECC000AAE029E000E78EF07F0010E10EC01F056
:100EDC0078EF07F0020E04EC01F078EF07F0040E47
:060EEC0017EC01F01200FA
:100EF2000501EC6BE9C5E9FFEAC5EAFFEECFEBF5C8
:100F0200EB51000A0EE0EBC5F0F535DD0501EC2BE7
:100F1200EC51E925E96E000EEA21EA6EEECFEBF51F
:040F2200EFD71200F3
:100F2600E9C5F6FFEAC5F7FFEBC5F8FF0900F5CFFF
:100F360000F0005211E0E9C5F6FFEAC5F7FFEBC580
:100F4600F8FF0900F5CFF0F539DD010E0501E927B7
:0A0F5600000EEA23EB23E4D712009B
:100F6000A39A0001CA6BCB6B010ECB5D02E1800E30
:100F7000CA5D0EE2490ECA25E16E020ECB21E26E79
:100F8000E1CFE1FFE2CFE2FFE66ACA4BCB2BECD721
:100F9000B46BB56BCA6BCB6BAACF7FF505017F6BCA
:0A0FA0000001B26BB36BA38A1200CC
:100FAA0000C008F00150006E016A026A036A0B6A07
:100FBA000C6A016A026A036A960E036E0A6A00AE36
:100FCA00EDEF07F0081E001E082AD8B4002A0A8E80
:100FDA0000C001F008C000F0086A026A42EC02F0A0
:020FEA001200F3
:080FEC00067EACEC02F01200DD
:100FF400000E0501EA1902E1000EE91935E0E9C520
:10100400E9FFEAC5EAFFEE522FE0EBC5F0F5ECC5C7
:10101400F1F5E0DC00C0F4F5E9C5F0F5EAC5F1F559
:10102400EBC5F2F5ECC5F3F57BEC02F0000E01180C
:1010340002E1000E001805E1E9C500F0EAC501F07F
:1010440015D0010E0501E925F06F000EEA21F16FBC
:10105400EBC5E9FFECC5EAFFEECFF2F592DC00C088
:0E106400E9F501C0EAF5C4D7006A016A12007E
:101072000D0E0501F06F7FDC0A0E0501F06F7BDCBF
:0210820012005A
:10108400E9C5F6FFEAC5F7FFEBC5F8FF0900F5CFA0
:1010940000F0005211E0E9C5F6FFEAC5F7FFEBC521
:1010A400F8FF0900F5CFF0F565DC010E0501E9272D
:0A10B400000EEA23EB23E4D712003C
:1010BE000B6A0A6A096A086A0E6A03340836045013
:1010CE00085E0550D8A0053C095E0650D8A0063C27
:1010DE000A5E0750D8A0073C0B5EE86AD8A0010E46
:1010EE000E5E0336070E0C6E0334083609360A36CA
:1010FE000B360E36045003A012D0085E0550D8A051
:10110E00053C095E0650D8A0063C0A5E0750D8A0E2
:10111E00073C0B5EE86AD8A0010E0E5E11D00826C1
:10112E000550D8B0053C09260650D8B0063C0A2614
:10113E000750D8B0073C0B26E86AD8B0010E0E2631
:10114E0003360C2ED1D70234083609360A360B3642
:10115E000E36045003A012D0085E0550D8A0053CF0
:10116E00095E0650D8A0063C0A5E0750D8A0073C80
:10117E000B5EE86AD8A0010E0E5E11D0082605504F
:10118E00D8B0053C09260650D8B0063C0A260750B2
:10119E00D8B0073C0B26E86AD8B0010E0E260236F0
:1011AE00070E0C6E0234083609360A360B360E362A
:1011BE00045002A012D0085E0550D8A0053C095E6E
:1011CE000650D8A0063C0A5E0750D8A0073C0B5E1E
:1011DE00E86AD8A0010E0E5E11D008260550D8B0D0
:1011EE00053C09260650D8B0063C0A260750D8B052
:1011FE00073C0B26E86AD8B0010E0E2602360C2EDE
:10120E00D1D70134083609360A360B360E3604505D
:10121E0002A012D0085E0550D8A0053C095E06500B
:10122E00D8A0063C0A5E0750D8A0073C0B5EE86AC1
:10123E00D8A0010E0E5E11D008260550D8B0053C80
:10124E0009260650D8B0063C0A260750D8B0073CEF
:10125E000B26E86AD8B0010E0E260136070E0C6E6C
:10126E000134083609360A360B360E36045001A004
:10127E0012D0085E0550D8A0053C095E0650D8A0D5
:10128E00063C0A5E0750D8A0073C0B5EE86AD8A061
:10129E00010E0E5E11D008260550D8B0053C092669
:1012AE000650D8B0063C0A260750D8B0073C0B268D
:1012BE00E86AD8B0010E0E2601360C2ED1D70034B6
:1012CE00083609360A360B360E36045001A012D0F7
:1012DE00085E0550D8A0053C095E0650D8A0063C15
:1012EE000A5E0750D8A0073C0B5EE86AD8A0010E34
:1012FE000E5E11D008260550D8B0053C09260650C2
:10130E00D8B0063C0A260750D8B0073C0B26E86A30
:10131E00D8B0010E0E260036070E0C6E00340836BD
:10132E0009360A360B360E36045000A012D0085E6F
:10133E000550D8A0053C095E0650D8A0063C0A5EB2
:10134E000750D8A0073C0B5EE86AD8A0010E0E5ECF
:10135E0011D008260550D8B0053C09260650D8B045
:10136E00063C0A260750D8B0073C0B26E86AD8B0D0
:10137E00010E0E2600360C2ED1D700B00ED0045022
:10138E0008260550D8B0053C09260650D8B0063CB4
:0C139E000A260750D8B0073C0B261200AE
:1013AA00DADDD2C5E9F5D3C5EAF5D4C5EBF5B6DD84
:1013BA00D2DD7A0E0B6EC10E0C6E810E0D6E0D2EE5
:1013CA00FED70C2EFCD70B2EFAD700000000050121
:1013DA00D55330E0490EE96F020EEA6F85DD490EFA
:1013EA00E96F020EEA6FC50EEB6F000EEC6FFDDDC2
:1013FA00000E026E0150025C02E10050000803E296
:10140A000301CB4BCC2BCBC3E9F5CCC3EAF547C2DE
:10141A00EBF548C2ECF570EC05F0A90EE96F4D0E3C
:10142A00EA6F000EEB6F29DE47C2E9F548C2EAF51A
:10143A005BDD1ADE19DE3D0E0B6EE10E0C6E3F0E01
:10144A000D6E0D2EFED70C2EFCD70B2EFAD70000F0
:04145A00000012007C
:10145E000501D56BD2C5E9FFD3C5EAFFEECFD4F5B2
:10146E00D451000A0FE0D4C5F0F5E1EC04F005010B
:10147E00D52BD551D225E96E000ED321EA6EEECFD3
:06148E00D4F5EED71200B8
:10149400220E0C6E086A096A0A6A0B6A0C06D8B432
:1014A4001FD0D8900B320A3209320832033202328A
:1014B40001320032D8A0F2D70C06D8B409D00450B7
:1014C40008260550092206500A2207500B22EAD7A3
:1014D400045008260550092206500A2207500B2200
:0214E4001200F4
:1014E6000050086E0150006E016A026A036A0B6AB8
:1014F6000C6A960E036E0A6A00C001F008C000F07E
:0A150600086A026A42EC02F01200CB
:10151000D2C504F0D3C505F00501D651D71124E09A
:10152000010ED65F000ED75B04C002F005C003F0C9
:10153000044A052AD4C500F0D5C501F0D44BD52BFB
:1015400000C0E9FF01C0EAFF02C0E1FF03C0E2FF03
:10155000EECFE6FF02C0E9FF03C0EAFFEECF00F0E6
:10156000005201E101D0D8D7D6C500F0D7C501F0AF
:10157000010ED65F000ED75B0050011008E004C0DA
:10158000E1FF05C0E2FFE66A044A052AEDD7D2C5AD
:0815900000F0D3C501F01200C8
:101598000501D851000805E3070ED96F000EDA6F70
:1015A80012D0D851160805E2170EDB6F000EDC6F5B
:1015B80006D0D851010FDB6FDC6B000EDC23DBC5D6
:1015C800D9F5DCC5DAF5D9C5E3F5DAC5E4F5DD6B9F
:1015D800DE6B046A056A066A076AD2C500F0D3C5DD
:1015E80001F0D4C502F0D5C503F009EC05F0010EF1
:1015F800D8B0000E006E005209E0D6C5E1FFD7C58D
:10160800E2FF2D0EE66ED64BD72BD47FD2C504F061
:10161800D3C505F0D4C506F0D5C507F0006A016A40
:10162800026A036A09EC05F0010ED8B0000E006EDC
:10163800005237E0000E046E000E056E000E066EB6
:101648007F0E076ED2C500F0D3C501F0D4C502F0F5
:10165800D5C503F009EC05F0010ED8B0000E006EF8
:1016680000521FE0D2C500F0D3C501F0D4C502F086
:10167800D5C503F0000E046E000E056E200E066E32
:10168800820E076EE6EC06F000C0D2F501C0D3F575
:1016980002C0D4F503C0D5F5010EDD5F000EDE5B98
:1016A800C9D7000E046E000E056E200E066E820E5F
:1016B800076ED2C500F0D3C501F0D4C502F0D5C578
:1016C80003F009EC05F0000ED8B0010E006E0052D0
:1016D8001EE0000E046E000E056E200E066E820ED1
:1016E800076ED2C500F0D3C501F0D4C502F0D5C548
:1016F80003F022EC06F000C0D2F501C0D3F502C019
:10170800D4F503C0D5F50501DD4BDE2BCAD7DD5175
:10171800E327DE51E423010EDF6F000EE06F000EB9
:10172800E56F000EE66F000EE76F7F0EE86F800E24
:10173800E019006E800EE419005C02E1E351DF5D00
:101748001EE2000E046E000E056E200E066E820E5E
:10175800076EE5C500F0E6C501F0E7C502F0E8C58B
:1017680003F022EC06F000C0E5F501C0E6F502C082
:10177800E7F503C0E8F50501DF4BE02BD8D7000EED
:10178800046E000E056E000E066E800E076EE5C52F
:1017980000F0E6C501F0E7C502F0E8C503F022EC69
:1017A80006F0D2C504F0D3C505F0D4C506F0D5C5FA
:1017B80007F0ACEC02F000C0D2F501C0D3F502C0CE
:1017C800D4F503C0D5F5000E046E000E056E200E8C
:1017D800066E820E076E09EC05F0000ED8B0010EF9
:1017E800006E00520BE0000E0501D26F000ED36FA1
:1017F800000ED46F7F0ED56FDD4BDE2B0501800EFA
:10180800DE19006E800E005C02E1000EDD5D38E23C
:10181800D6C5E1FFD7C5E2FF300EE66ED64BD72B13
:10182800D6C5E1FFD7C5E2FF2E0EE66ED64BD72B05
:10183800800EE419006E800E005C02E1000EE35D8C
:1018480004E2E351DD5FE451DE5BFF0EDF6FFF0E64
:10185800E06F800EDE19006E800EE019005C02E178
:10186800DF51DD5D0DE2D6C5E1FFD7C5E2FF300EE1
:10187800E66ED64BD72B010EDF5F000EE05BE9D793
:10188800DF6BE06B800EE019006E800EE419005CDF
:1018980002E1E351DF5D63E2D2C500F0D3C501F098
:1018A800D4C502F0D5C503F0B9EC05F000C0E1F5E8
:1018B80001C0E2F5300E0026D6C5E1FFD7C5E2FF2C
:1018C80000C0E6FFD64BD72BE051DE1902E1DD510F
:1018D800DF1908E1D6C5E1FFD7C5E2FF2E0EE66E97
:1018E800D64BD72BE1C500F0E2C501F0D5EC07F0E7
:1018F80000C0E5F501C0E6F502C0E7F503C0E8F56C
:1019080000C004F001C005F002C006F003C007F0F3
:10191800D2C500F0D3C501F0D4C502F0D5C503F097
:10192800F6EC07F000C0D2F501C0D3F502C0D4F53B
:1019380003C0D5F5000E046E000E056E200E066E6F
:10194800820E076EE6EC06F000C0D2F501C0D3F5B2
:1019580002C0D4F503C0D5F5DF4BE02B93D7D6C52D
:0A196800E1FFD7C5E2FFE66A1200B6
:10197200D2C504F0D3C505F004C0E9FF05C0EAFFF3
:10198200EE5203E0044A052AF7D704C002F005C06C
:1019920003F0044A052AD4C500F0D5C501F00501BB
:1019A200D44BD52B00C0E9FF01C0EAFF02C0E1FF22
:1019B20003C0E2FFEECFE6FF02C0E9FF03C0EAFF89
:1019C200EE5201E0E2D7D2C500F0D3C501F0120019
:1019D200D4C5F6FFD5C5F7FFD6C5F8FF0900F5CF88
:1019E20000F0005218E0D4C5F6FFD5C5F7FFD6C502
:1019F200F8FF0900F5CF00F0D2C5E1FFD3C5E2FF41
:101A020000C0E6FF0501D24BD32B010ED427000EF6
:101A1200D523D623DDD7D2C5E1FFD3C5E2FFE66ADF
:021A22001200B0
:101A2400C26A070EC16EC18ED2C500F000360090A6
:101A3400003600900050C212C280DFEC06F0C28271
:101A4400C2A201D0FDD7C4CF01F0006AC350001276
:081A5400000E0112C290120005
:101A5C000900F5CFE6FF0006FBE10106F9E11200F3
:101A6C00FF0E01018B6FFF0E8C6FFF0E8D6FFF0E43
:0E1A7C008E6FC26A070EC16EC18EC28012004C
:101A8A0080C504F081C505F004C002F005C003F06A
:101A9A00044A052A82C500F083C501F00501824B7C
:101AAA00832B00C0E9FF01C0EAFF02C0E1FF03C0C7
:101ABA00E2FFEECFE6FF02C0E9FF03C0EAFFEE5203
:0E1ACA0001E0E2D780C500F081C501F01200F6
:101AD8000501866B876B000E875D02E10A0E865D45
:101AE8000BE286518425E16E87518521E26E200E36
:101AF800E66E864B872BEFD786518425E16E87519A
:101B08008521E26EE66A010E865F000E875B8651CC
:101B18008425886F87518521896F0A0E046E000E0F
:101B2800056E066E076E80C500F081C501F082C59E
:101B380002F083C503F05FEC08F008C000F009C0AC
:101B480001F00AC002F00BC003F0300E002688C571
:101B5800E1FF89C5E2FF00C0E6FF0A0E046E000E31
:101B6800056E066E076E80C500F081C501F082C55E
:101B780002F083C503F05FEC08F000C080F501C0F7
:101B880081F502C082F503C083F5000E046E0318C8
:101B980008E10450021805E10450011802E1005060
:101BA800000A01E105D0010E865F000E875BAFD702
:021BB800120019
:101BBA00FF0E986EEF0E926EBF0E946EC088F90EED
:101BCA00C16EFF0EC26EC0989380938492809594E2
:101BDA00938093969596F19E9A8A92988988958E83
:0E1BEA00998695989698959C8C988D981200E7
:101BF800780E0101976F090E986FF00E996F050E18
:101C08009A6FFF0E9B6FFF0E9C6F000E9D6F000E6C
:101C18009E6FFF0E9F6FFF0EA06F000EA16F000E4C
:101C2800A26FFF0E8F6FFF0E906F000E916F000E68
:101C3800926FAD8A900EAC6E948E949C9EAA03D03F
:081C4800AFCF00F0FBD7120042
:101C5000C20E0101976F090E986FF00E996F050E75
:101C60009A6FFF0E9B6FFF0E9C6F000E9D6F000E14
:101C70009E6FFF0E9F6FFF0EA06F000EA16F000EF4
:101C8000A26FFF0E8F6FFF0E906F000E916F000E10
:101C9000926FA88A900E9C6E98849892A4AA03D002
:081CA000AACF00F0FBD71200EF
:101CA800810E0501E96F490EEA6F000EEB6F42ECF9
:101CB80008F080C5E9F581C5EAF579EC07F039EC5B
:101CC80008F0B0EC07F0900E0501E96F4C0EEA6FD2
:101CD800000EEB6F42EC08F005014D6B4D0ED26F14
:101CE800050ED36FD90ED46F4D0ED56F000ED66F7B
:101CF8006CDE550E0501D26F050ED36F0F0E006E08
:101D0800000E016E026E036E7DC504F07EC505F0FF
:101D1800000E7EBFFF0E066E076E4AEC0AF0EF0E4D
:101D28000024D46F450E0120D56F000E0220D66F17
:101D38004CDE4D0E0501E96F050EEA6F79EC07F0F0
:101D480039EC08F0B0EC07F04D0E0501D26F050E26
:101D5800D36F2FEC0AF00D0EF06FE1EC04F0F40EE7
:101D68000B6E820E0C6E050E0D6E0D2EFED70C2E10
:101D7800FCD70B2EFAD739EC08F0490E0501E96FAC
:101D8800020EEA6FC00EEB6F000EEC6FFAEC07F074
:101D980000C0C9F301C0CAF3000E026E0150025C14
:101DA80002E100500008D8B093D0B0EC07F0490E1B
:101DB8000501E96F4A0EEA6F000EEB6F42EC08F07E
:101DC80080C5D2F581C5D3F52FEC0AF01A0EF06F55
:101DD800E1EC04F00D0E0501F06FE1EC04F0020EE9
:101DE8000A6E120E0B6EF20E0C6E240E0D6E0D2E78
:101DF800FED70C2EFCD70B2EFAD70A2EF8D70000E8
:101E0800490E0501E96F020EEA6F79EC07F0490EF9
:101E1800E96F020EEA6FBD0EEB6F000EEC6FFAEC85
:101E280007F000C0C9F301C0CAF3000E026E0150EA
:101E3800025C02E10050000841E2A70E0201476F70
:101E4800010E486FD30E0501E96F4C0EEA6F000EC4
:101E5800EB6F42EC08F0490E0501E96F020EEA6FDC
:101E6800B60EEB6F000EEC6FFAEC07F000C0C9F38A
:101E780001C0CAF347C2D2F548C2D3F500C0D4F5B1
:101E880001C0D5F50A0E0501D66F000ED76F88EC94
:101E98000AF047C2E9F548C2EAF579EC07F039ECEF
:101EA80008F0100E0301C925E16E000ECA21E26E8A
:101EB800E1CFE1FFE2CFE2FFE66A09D07E0E05013D
:101EC800E96F4A0EEA6F000EEB6F42EC08F009D09A
:101ED800B20E0501E96F4C0EEA6F000EEB6F42EC93
:0C1EE80008F039EC08F0B0EC07F0120034
:101EF4009D989D9A0001C86BC96B010EC95D02E1F2
:101F0400800EC85D0EE2CD0EC825E16E030EC92118
:101F1400E26EE1CFE1FFE2CFE2FFE66AC84BC92BF4
:101F2400ECD7C86BC96BCC6BCD6BAFCFC2F0C26BB7
:081F3400C36BC46B9D8A12000F
:101F3C0080C5E1FF81C5E2FFE66A0501826B80C5C1
:101F4C00D2F581C5D3F50C0ED46F4B0ED56F000EA8
:101F5C00D66F39DD80C5F0F581C5F1F5ECEC04F0F8
:101F6C0000C0C8F001C0C9F0826B820ED26F050EA2
:101F7C00D36F140ED46F4E0ED56F000ED66F23DDBB
:101F8C00820E0501F06F050EF16FECEC04F000C051
:101F9C00C8F001C0C9F0820E0024E16E050E0120CC
:101FAC00E26E006A83BE002A300E0026E1CFE1FF0C
:101FBC00E2CFE2FF00C0E6FF0001C84BC92B820E46
:101FCC00C825E16E050EC921E26EE1CFE1FFE2CF3B
:101FDC00E2FF0D0EE66EC84BC92B820EC825E16ED2
:101FEC00050EC921E26EE1CFE1FFE2CFE2FF0A0E5E
:101FFC00E66EC84BC92B820EC825E16E050EC921B1
:10200C00E26EE1CFE1FFE2CFE2FFE66A80C5D2F5F6
:10201C0081C5D3F5820E0501D46F050ED56FA3DCF7
:10202C00826B820ED26F050ED36F040ED46F4E0EE0
:10203C00D56F000ED66FC7DC820E0501F06F050E52
:10204C00F16FECEC04F000C0C8F001C0C9F0820ED6
:10205C000024E16E050E0120E26E006A87B6002AAC
:10206C00300E0026E1CFE1FFE2CFE2FF00C0E6FF39
:10207C000001C84BC92B820EC825E16E050EC92183
:10208C00E26EE1CFE1FFE2CFE2FF0D0EE66EC84B50
:10209C00C92B820EC825E16E050EC921E26EE1CF77
:1020AC00E1FFE2CFE2FF0A0EE66EC84BC92B820EAF
:1020BC00C825E16E050EC921E26EE1CFE1FFE2CF4A
:1020CC00E2FFE66A80C5D2F581C5D3F5820E050123
:1020DC00D46F050ED56F47DC826B820ED26F050E66
:1020EC00D36F1C0ED46F4E0ED56F000ED66F6BDCFB
:1020FC00820E0501F06F050EF16FECEC04F000C0E0
:10210C00C8F001C0C9F0820E0024E16E050E01205A
:10211C00E26E006A83B8002A300E0026E1CFE1FFA0
:10212C00E2CFE2FF00C0E6FF0001C84BC92B820ED4
:10213C00C825E16E050EC921E26EE1CFE1FFE2CFC9
:10214C00E2FF0D0EE66EC84BC92B820EC825E16E60
:10215C00050EC921E26EE1CFE1FFE2CFE2FF0A0EEC
:10216C00E66EC84BC92B820EC825E16E050EC9213F
:10217C00E26EE1CFE1FFE2CFE2FFE66A80C5D2F585
:10218C0081C5D3F5820E0501D46F050ED56FB9EC60
:10219C000CF0826B820ED26F050ED36F3C0ED46F97
:1021AC004E0ED56F000ED66F0EDC820E0501F06F51
:1021BC00050EF16FECEC04F000C0C8F001C0C9F0E2
:1021CC00820E0024E16E050E0120E26E006A84B8D6
:1021DC00002A300E0026E1CFE1FFE2CFE2FF00C083
:1021EC00E6FF0001C84BC92B820EC825E16E050E17
:1021FC00C921E26EE1CFE1FFE2CFE2FF0D0EE66E08
:10220C00C84BC92B820EC825E16E050EC921E26EA2
:10221C00E1CFE1FFE2CFE2FF0A0EE66EC84BC92B1D
:10222C00820EC825E16E050EC921E26EE1CFE1FFF9
:10223C00E2CFE2FFE66A80C5D2F581C5D3F5820E06
:10224C000501D46F050ED56FB9EC0CF0826B010E45
:10225C00D26F12EC0DF000C02EF101C02FF1015025
:10226C00020802E1005000080EE2820E0501D26F56
:10227C00050ED36F100ED46F4D0ED56F000ED66FAA
:10228C00E9EC0CF00DD0820E0501D26F050ED36F68
:10229C00810ED46F4E0ED56F000ED66FE9EC0CF09C
:1022AC00820E0501F06F050EF16FECEC04F000C02E
:1022BC00C8F001C0C9F02EC1E9F52FC1EAF5820EB4
:1022CC000024EB6F050E0120EC6F70EC05F0820E14
:1022DC00F06F050EF16FECEC04F000C0C8F001C01B
:1022EC00C9F0820E0024E16E050E0120E26EE1CFF2
:1022FC00E1FFE2CFE2FF0D0EE66E0001C84BC92BE9
:10230C00820EC825E16E050EC921E26EE1CFE1FF18
:10231C00E2CFE2FF0A0EE66EC84BC92B820EC8252F
:10232C00E16E050EC921E26EE1CFE1FFE2CFE2FFE3
:10233C00E66A80C5D2F581C5D3F5820E0501D46F4E
:10234C00050ED56FB9EC0CF0826B30C104F031C1C5
:10235C0005F032C106F033C107F0000E006E000E1E
:10236C00016E280E026E830E036E09EC05F0010E51
:10237C00D8B0000E006E00520DE0820ED26F050E2A
:10238C00D36F020ED46F4D0ED56F000ED66FE9ECE5
:10239C000CF00DD0820E0501D26F050ED36F0C0E12
:1023AC00D46F4E0ED56F000ED66FE9EC0CF0820E8A
:1023BC000501F06F050EF16FECEC04F000C0C8F0F5
:1023CC0001C0C9F030C1D2F531C1D3F532C1D4F559
:1023DC0033C1D5F5820E0024D66F050E0120D76FC0
:1023EC00020ED86FCCEC0AF0820EF06F050EF16F76
:1023FC00ECEC04F000C0C8F001C0C9F0820E00245F
:10240C00E16E050E0120E26EE1CFE1FFE2CFE2FFCB
:10241C005F0EE66E0001C84BC92B820EC825E16E1B
:10242C00050EC921E26EE1CFE1FFE2CFE2FF430EE0
:10243C00E66EC84BC92B820EC825E16E050EC9216C
:10244C00E26EE1CFE1FFE2CFE2FFE66A80C5D2F5B2
:10245C0081C5D3F5820E0501D46F050ED56FB9EC8D
:10246C000CF0826B820ED26F050ED36F8B0ED46F75
:10247C004D0ED56F000ED66FE9EC0CF080C5D2F581
:10248C0081C5D3F5820E0501D46F050ED56FB9EC5D
:10249C000CF0826B80C5F0F581C5F1F5ECEC04F025
:0A24AC0000C0C8F001C0C9F0120022
:1024B600D596D584D582D580D59AD59C480ED76E2B
:1024C600E50ED66EF29401012C6B2D6B876B886B33
:0824D600F184F28AD58E120098
:1024DE000501806B816B316A326AD00EE96F4B0E4B
:1024EE00EA6F000EEB6F42EC08F0B0EC07F0A50EB1
:1024FE000501E96F4E0EEA6F000EEB6F93EC07F0DD
:10250E003D0E0B6EE10E0C6E3F0E0D6E0D2EFED7B8
:10251E000C2EFCD70B2EFAD700000000000E000187
:10252E00B31902E1010EB21922E1490E0501E96F5C
:10253E00020EEA6F2E0EEB6F000EEC6FFAEC07F048
:10254E00000E026E0150025C02E1005000080FE224
:10255E00150E0501806F000E816F010E316E000E9B
:10256E00326E490EE96F020EEA6F79EC07F01F0E1C
:10257E000B6E710E0C6E1E0E0D6E05010D2EFDD71F
:10258E000C2EFBD70B2EF9D70000804B812B800E23
:10259E008119006E800E005C02E1140E805D07E270
:1025AE00000E321802E1000E311801E19ED7120022
:1025BE008D88010E0301CB6F000ECC6F010189894E
:1025CE00A00E0501E96F490EEA6F000EEB6F42ECAB
:1025DE0008F0BD0E0501D26F4D0ED36F000ED46FF5
:1025EE00000E010189B9010E0501D56FD5EC09F078
:1025FE00590E0501E96F430EEA6F000EEB6F42ECC8
:10260E0008F0E30E0501D26F4C0ED36F000ED46F9F
:10261E00000E010189B9010E0501D56FD5EC09F047
:10262E00C60E0501E96F460EEA6F000EEB6F42EC27
:10263E0008F0800E0501D26F4D0ED36F000ED46FD1
:10264E00000E010189B9010E0501D56FD5EC09F017
:10265E00E60E0501E96F480EEA6F000EEB6F42ECD5
:10266E0008F0B30E0501D26F4D0ED36F000ED46F6E
:10267E00000E010189B9010E0501D56FD5EC09F0E7
:10268E00650E0501E96F480EEA6F000EEB6F42EC26
:10269E0008F0E20E0501D26F4D0ED36F000ED46F0F
:1026AE00000E010189B9010E0501D56FD5EC09F0B7
:1026BE00190E0501E96F470EEA6F000EEB6F42EC43
:1026CE0008F09F0E0501D26F4E0ED36F000ED46F21
:1026DE00000E010189B9010E0501D56FD5EC09F087
:1026EE00B20E0501E96F470EEA6F000EEB6F42EC7A
:1026FE0008F0AF0E0501D26F4A0ED36F000ED46FE5
:10270E00000E010189B9010E0501D56FD5EC09F056
:10271E00720E0501E96F460EEA6F000EEB6F42EC8A
:10272E0008F01E0E0501D26F4D0ED36F000ED46F42
:10273E00000E010189B9010E0501D56FD5EC09F026
:10274E00190E0501E96F430EEA6F000EEB6F42ECB6
:10275E0008F01C0E0501D26F460ED36F000ED46F1B
:10276E00000E010189B9010E0501D56FD5EC09F0F6
:10277E00D70E0501E96F420EEA6F000EEB6F42ECC9
:10278E0008F0C20E0501D26F450ED36F000ED46F46
:10279E00000E010189B9010E0501D56FD5EC09F0C6
:1027AE001F0E0501E96F480EEA6F000EEB6F42EC4B
:1027BE0008F09F0E0501D26F4D0ED36F000ED46F31
:1027CE00000E010189B9010E0501D56FD5EC09F096
:1027DE00410E0501E96F470EEA6F000EEB6F42ECFA
:1027EE0008F05D0E0501D26F4D0ED36F000ED46F43
:1027FE00000E010189B9010E0501D56FD5EC09F066
:10280E00C70E0501E96F4A0EEA6F000EEB6F42EC40
:10281E0008F0870E0501D26F4E0ED36F000ED46FE7
:10282E00000E010189B9010E0501D56FD5EC09F035
:10283E009C0E0501E96F460EEA6F000EEB6F42EC3F
:10284E0008F0750E0501D26F4D0ED36F000ED46FCA
:10285E00000E010189B9010E0501D56FD5EC09F005
:10286E004E0E0501E96F420EEA6F000EEB6F42EC61
:10287E0008F0BD0E0501D26F490ED36F000ED46F56
:10288E00000E010189B9010E0501D56FD5EC09F0D5
:10289E00F00E0501E96F460EEA6F000EEB6F42EC8B
:1028AE0008F0950E0501D26F4D0ED36F000ED46F4A
:1028BE00000E010189B9010E0501D56FD5EC09F0A5
:1028CE00D00E0501E96F430EEA6F000EEB6F42EC7E
:1028DE0008F0B0EC07F0220E0501E96F4B0EEA6F1F
:1028EE00000EEB6F93EC07F0D60E0B6E110E0C6E06
:1028FE00E40E0D6E0D2EFED70C2EFCD70B2EFAD736
:10290E000000490E0501E96F020EEA6F79EC07F03F
:10291E0039EC08F08D0E0501E96F470EEA6F000ED7
:10292E00EB6F42EC08F0210E0501D26F4C0ED36F07
:10293E00000ED46F000E010189B9010E0501D56F8D
:10294E00D5EC09F0420E0501E96F480EEA6F000E54
:10295E00EB6F42EC08F0F40E0501D26F4D0ED36F03
:10296E00000ED46F000E010189B9010E0501D56F5D
:10297E00D5EC09F0430E0501E96F490EEA6F000E22
:10298E00EB6F42EC08F0380E0501D26F4D0ED36F8F
:10299E00000ED46F000E010189B9010E0501D56F2D
:1029AE00D5EC09F05C0E0B6E510E0C6E600E0D6EBA
:1029BE000D2EFED70C2EFCD70B2EFAD700005A0E7A
:1029CE000501E96F4C0EEA6F000EEB6F42EC08F05A
:1029DE00CBC3E9F5CCC3EAF547C2EBF548C2ECF53B
:1029EE0070EC05F047C2E9F548C2EAF579EC07F05C
:1029FE002C0EE96F4E0EEA6F000EEB6F42EC08F0F4
:0A2A0E00CBC300F0CCC301F01200AE
:102A18000101346B356B1A6B1B6B000E1B5D02E1F9
:102A2800080E1A5D18E21AC100F01BC101F0003649
:102A3800009001361C0E0024D96E010E0120DA6EBA
:102A4800D9CFD9FFDACFDAFFDE503427DE5035236D
:102A58001A4B1B2BE2D734C100F035C101F073ECDF
:102A68000AF0000E046E000E056E250E066E7A0E34
:082A7800076EE6EC06F0120007
:102A800055EC27F0DDEC0DF08D88A70E0201476FA5
:102A9000010E486F0101A76B366B0201496B010102
:102AA0002E6B2F6B866B186B196B866B010E0001FA
:102AB000D46F010ED56F0301CB6BCC6B01018989FB
:102AC0008997899D8A81899F89938C9C05017D6B5B
:102AD0007E6B8D988C887E86020E7F6E700EB06E37
:102AE000AD84FCEC0DF01F0E0B6E710E0C6E1E0E05
:102AF0000D6E0D2EFED70C2EFCD70B2EFAD7000034
:102B000039EC08F08C987C86020E7D6E700EAB6EF0
:102B1000A88428EC0EF0070E0B6E170E0C6E6A0ED2
:102B20000D6E0D2EFED70C2EFCD70B2EFAD7000003
:102B3000010E0501E96F420EEA6F000EEB6F42ECE9
:102B400008F0B20E0501E96F410EEA6F000EEB6F5F
:102B500042EC08F0630E0501E96F410EEA6F000ECA
:102B6000EB6F42EC08F0070E0501E96F440EEA6FC7
:102B7000000EEB6F42EC08F0040E0501E96F450E04
:102B8000EA6F000EEB6F42EC08F0D20E0501E96F20
:102B9000440EEA6F000EEB6F42EC08F0C70E050121
:102BA000E96F4D0EEA6F000EEB6F42EC08F0800EFD
:102BB0000001D66FBB0ED76F000ED86FD96F800E95
:102BC0000501806FBB0E816F000E826F000E836F58
:102BD00047C284F548C285F56CEC0DF047C2E9F5B3
:102BE00048C2EAF579EC07F039EC08F0F30E05017C
:102BF000E96F4C0EEA6F000EEB6F42EC08F0930E9B
:102C00000501E96F420EEA6F000EEB6F42EC08F02F
:102C1000BB0E0501E96F400EEA6F000EEB6F42EC50
:102C200008F0130E0501E96F410EEA6F000EEB6F1D
:102C300042EC08F07A0E0501E96F4B0EEA6F000EC8
:102C4000EB6F42EC08F0EF0E0501E96F450EEA6FFD
:102C5000000EEB6F42EC08F039EC08F0FE0E0501B7
:102C6000E96F450EEA6F000EEB6F42EC08F039ECAD
:102C700008F039EC08F036EC0DF02B0E0501E96F89
:102C80004D0EEA6F000EEB6F42EC08F0980E050156
:102C9000E96F430EEA6F000EEB6F42EC08F0FB0E9B
:102CA0000501E96F470EEA6F000EEB6F42EC08F08A
:102CB000010E0501D26F12EC0DF000C02EF101C023
:102CC0002FF100C0E9F501C0EAF547C2EBF548C2B3
:102CD000ECF570EC05F047C2E9F548C2EAF579EC8D
:102CE00007F0090EF06FBCEC04F00101346B356B9A
:102CF000020E0501D26F12EC0DF000C0CEF001C043
:102D0000CFF000C0E9F501C0EAF547C2EBF548C2D3
:102D1000ECF570EC05F047C2E9F548C2EAF579EC4C
:102D200007F039EC08F0020E0501D26F12EC0DF03D
:102D300000C0CEF001C0CFF001011A6B1B6B000E7A
:102D40001B5D02E1080E1A5D18E21AC100F01BC1FA
:102D500001F00036009001361C0E0024E16E010ED9
:102D60000120E26EE1CFE1FFE2CFE2FFCEC0E6FF5D
:102D7000CFC0E6FF1A4B1B2BE2D70001D06BD16B03
:102D8000860E0501E96F480EEA6F000EEB6F42EC0C
:102D900008F03D0E0B6EE10E0C6E3F0E0D6E0D2E0B
:102DA000FED70C2EFCD70B2EFAD7000000008C9417
:102DB000B70E0B6EA10E0C6EC30E0D6E0D2EFED750
:102DC0000C2EFCD70B2EFAD7000000008C843D0E91
:102DD0000B6EE10E0C6E3F0E0D6E0D2EFED70C2EFF
:102DE000FCD70B2EFAD7000000008C96F50E0501DB
:102DF000E96F4A0EEA6F000EEB6F42EC08F0B0ECA0
:102E000007F0AC8EAC86AC969C96D08EA38AF28CE2
:102E1000F28E6FEC12F0000E321802E1010E311842
:102E20000AE17E0E0501E96F4C0EEA6F000EEB6FB2
:102E300042EC08F022D0620E0501E96F490EEA6FFC
:102E4000000EEB6F42EC08F0A00E0501E96F440E96
:102E5000EA6F000EEB6F42EC08F08C783D0E0B6EC3
:102E6000E10E0C6E3F0E0D6E0D2EFED70C2EFCD714
:102E70000B2EFAD700000000F0D7A70E0201476F13
:102E8000010E486F2E0E0501E96F4A0EEA6F000E23
:102E9000EB6F42EC08F0DFEC12F000C0CBF301C0A6
:102EA000CCF3800E026E800E0118025C02E100502D
:102EB00012080CE2750E0501E96F4E0EEA6F000E66
:102EC000EB6F42EC08F0010189870BD0520E05012F
:102ED000E96F4E0EEA6F000EEB6F42EC08F0010155
:102EE000898739EC08F07A0E0B6EC10E0C6E810EDC
:102EF0000D6E0D2EFED70C2EFCD70B2EFAD7000030
:102F000000008C98A70E0201476F010E486F470E14
:102F10000501E96F460EEA6F000EEB6F42EC08F018
:102F200047C280F548C281F59EEC0FF000C0D2F098
:102F300001C0D3F039EC08F0070E0B6E170E0C6EC3
:102F40006A0E0D6E0D2EFED70C2EFCD70B2EFAD767
:102F500000008D980301CB6BCC6B01018999899D91
:102F60008C9CDE0E0501E96F4A0EEA6F000EEB6FD6
:102F700042EC08F07AEC0FF00101166B176BA70E0C
:102F80000201476F010E486F81B413D047C2D2F5DA
:102F900048C2D3F5240E0501D46F490ED56F000E3B
:102FA000D66FE9EC0CF047C280F548C281F554ECCD
:102FB0000EF001018A910001D06BD16BA70E0201C6
:102FC000476F010E486F7AEC0FF05BEC12F089ABA3
:102FD00000D0020E0501D26F12EC0DF0060E005C5F
:102FE000056E000E0158066E05C0CEF006C0CFF08B
:102FF000070E0001D015036ED1C004F0000E0416B8
:1030000003C000F004C001F00036009001361C0E31
:103010000024E16E010E0120E26EE1CFE1FFE2CF7C
:10302000E2FF05C0E6FF06C0E6FFD04BD12B010E44
:103030000501D26F12EC0DF000C02EF101C02FF18E
:10304000000E006E0001D151005C02E1D051080871
:1030500002E201018A810101000E191902E1000E4C
:103060001819D8A419D116C1E9F517C1EAF5360E19
:103070000501EB6F010EEC6F70EC05F0360EE96F99
:10308000010EEA6F79EC07F02EC1E9F52FC1EAF5E0
:10309000360EEB6F010EEC6F70EC05F0990EE96FD8
:1030A0004E0EEA6F000EEB6F42EC08F0360E050193
:1030B000E96F010EEA6F79EC07F04B0EE96F4E0EE7
:1030C000EA6F000EEB6F42EC08F0CEC0E9F5CFC01E
:1030D000EAF5360E0501EB6F010EEC6F70EC05F0B2
:1030E000360EE96F010EEA6F79EC07F0016A010113
:1030F0008AB1012A0150000832E28EDC00C030F1B2
:1031000001C031F102C032F103C033F1EB0E050111
:10311000E96F4D0EEA6F000EEB6F42EC08F030C124
:10312000D2F531C1D3F532C1D4F533C1D5F5360E60
:103130000501D66F010ED76F020ED86FCCEC0AF0E6
:10314000360EE96F010EEA6F79EC07F08D0EE96F2C
:103150004E0EEA6F000EEB6F42EC08F009D0C30E82
:103160000501E96F4C0EEA6F000EEB6F42EC08F0C0
:10317000930E0501E96F4E0EEA6F000EEB6F42EC05
:1031800008F0000E83BE010E0501F06F300EF0272F
:10319000BCEC04F0440E0501E96F4E0EEA6F000E20
:1031A000EB6F42EC08F0000E87B6010E0501F06FE0
:1031B000300EF027BCEC04F0590E0501E96F4E0EFD
:1031C000EA6F000EEB6F42EC08F0000E83B8010EC0
:1031D0000501F06F300EF027BCEC04F06E0E050117
:1031E000E96F4E0EEA6F000EEB6F42EC08F0000E36
:1031F00084B8010E0501F06F300EF027BCEC04F02E
:10320000D00E0501E96F4D0EEA6F000EEB6F42EC38
:1032100008F0000E010189B7010E0501F06F300EB4
:10322000F027BCEC04F0600E0501E96F4E0EEA6F6A
:10323000000EEB6F42EC08F0000E010189BD010E9B
:103240000501F06F300EF027BCEC04F0240E0501F0
:10325000E96F4E0EEA6F000EEB6F42EC08F0000EC5
:1032600080B0010E0501F06F300EF027BCEC04F0C9
:10327000670E0501E96F4E0EEA6F000EEB6F42EC30
:1032800008F0000E83BC010E0501F06F300EF02730
:10329000BCEC04F039EC08F00001D451010A08E15B
:1032A00001012F51020802E12E510008D8A08681A9
:1032B0000001D551010A1AE130C104F031C105F015
:1032C00032C106F033C107F0000E006E000E016E31
:1032D000280E026E830E036E09EC05F0010ED8B0C5
:1032E000000E006E005202E001018683010189BFD9
:1032F00008D08651000805E383AE03D087A601D02D
:10330000B9D089AD75D08C9CA70E0201476F010E14
:10331000486F47C2D2F548C2D3F5A10E0501D46F5C
:103320004C0ED56F000ED66FE9EC0CF047C2E9F5F4
:1033300048C2EAF579EC07F039EC08F05C0E0B6E48
:10334000510E0C6E600E0D6E0D2EFED70C2EFCD79E
:103350000B2EFAD70000670E0501E96F470EEA6FE2
:10336000000EEB6F42EC08F0510E0501D26F4D0ECE
:10337000D36F000ED46F000E010189B9010E050153
:10338000D56FD5EC09F07A0E0B6EC10E0C6E810E66
:103390000D6E0D2EFED70C2EFCD70B2EFAD700008B
:1033A00000006D0E0501E96F440EEA6F000EEB6F31
:1033B00042EC08F0900E0501D26F4B0ED36F000E59
:1033C000D46F000E010189B9010E0501D56FD5EC4E
:1033D00009F01F0E0B6E710E0C6E1E0E0D6E0D2E73
:1033E000FED70C2EFCD70B2EFAD700000101899DC9
:1033F000340E0501E96F4C0EEA6F000EEB6F42ECE4
:1034000008F047C280F548C281F59EEC0FF000C07D
:10341000D2F001C0D3F000C0E9F501C0EAF5360EE4
:10342000EB6F010EEC6F70EC05F0360EE96F010EDC
:10343000EA6F79EC07F039EC08F047C280F548C232
:1034400081F554EC0EF00101865304E0FE0E861760
:103450000001D46B0101865304E0FD0E86170001C4
:10346000D56B010189AF02D0899FF288B0EC07F0DB
:103470007AEC0FF00001000EB31902E1010EB2194F
:10348000D8A4D5EF1EF0010189BDD5EF1EF0490E7D
:103490000501E96F020EEA6F240EEB6F000EEC6F70
:1034A000FAEC07F000C0C9F301C0CAF3000E026EC7
:1034B0000150025C02E100500008D8B0C3D0640E95
:1034C0000501E96F450EEA6F000EEB6F42EC08F064
:1034D0004E0E0501E96F4B0EEA6F000EEB6F93EC99
:1034E00007F0D60E0B6E110E0C6EE40E0D6E0D2E47
:1034F000FED70C2EFCD70B2EFAD70000490E050183
:10350000E96F020EEA6F79EC07F039EC08F005017B
:103510007D6B7E6B490EE96F020EEA6F290EEB6F31
:10352000000EEC6FFAEC07F0000E026E0150025C28
:1035300002E10050000803E205017D6B7E6B05018E
:10354000490EE96F020EEA6F1A0EEB6F000EEC6F78
:10355000FAEC07F0000E026E0150025C02E100502E
:10356000000805E2010E05017D6F000E7E6F05016A
:10357000490EE96F020EEA6F1F0EEB6F000EEC6F43
:10358000FAEC07F000C0C9F301C0CAF3000E026EE6
:103590000150025C02E10050000854E2DA0E05011D
:1035A000D26F000ED36FC60ED46F480ED56F000ECB
:1035B000D66FE9EC0CF0E30E0501D26F000ED36F6D
:1035C000040E0301C9250501D46F000E0301CA21B1
:1035D0000501D56F0E0ED66F000ED76F88EC0AF07E
:1035E0000D0EE96F4C0EEA6F000EEB6F42EC08F027
:1035F000DA0E0501E96F000EEA6F79EC07F039EC9D
:1036000008F0B0EC07F0DA0E0501D26F000ED36FB0
:103610002FEC0AF0B70E0B6EA10E0C6EC30E0D6EE2
:103620000D2EFED70C2EFCD70B2EFAD70000000073
:10363000490EE96F020EEA6F79EC07F039EC08F0F9
:10364000B0EC07F0490E0501E96F020EEA6F330E88
:10365000EB6F000EEC6FFAEC07F000C0C9F301C08D
:10366000CAF3000E026E0150025C02E10050000835
:10367000D8B0A6D00101366B450E0501E96F4D0E9D
:10368000EA6F000EEB6F42EC08F0360E0501D26FC8
:10369000010ED36F050E0301C9250501D46F000E7D
:1036A0000301CA210501D56F080ED66F000ED76F32
:1036B00088EC0AF0360EE96F010EEA6F79EC07F03C
:1036C0000001D26BD36B800E0101A36F000EA46FBB
:1036D000A56BA66B1A6B1B6B000E1B5D02E1080E3F
:1036E0001A5D38E2360E1A25E96E010E1B21EA6ECC
:1036F000E9CFE9FFEACFEAFFEE50300A0EE0360EDE
:103700001A25E96E010E1B21EA6EE9CFE9FFEACF27
:10371000EAFFEE50310A01E003D00001D24BD32B77
:10372000360E01011A25E96E010E1B21EA6EE9CF62
:10373000E9FFEACFEAFFEE50310A04E1A351A527E1
:10374000A451A623A433A333A49FA4BDA48F1A4BD2
:103750001B2BC2D7000E0001D31902E1080ED219AB
:1037600017E1010189AB14D047C2D2F548C2D3F5A5
:10377000470E0501D46F4C0ED56F000ED66FE9ECE5
:103780000CF047C280F548C281F554EC0EF016D01B
:10379000010189AB0AD0350E0501E96F450EEA6FCC
:1037A000000EEB6F42EC08F009D0050E0501E96F41
:1037B000490EEA6F000EEB6F42EC08F0B0EC07F038
:1037C000490E0501E96F020EEA6F7E0EEB6F000EE7
:1037D000EC6FFAEC07F000C0C9F301C0CAF3000EA9
:1037E000026E0150025C02E1005000080DE201018E
:1037F0008997640E0501E96F4B0EEA6F000EEB6FBF
:1038000042EC08F0B0EC07F0490E0501E96F020E3A
:10381000EA6F610EEB6F000EEC6FFAEC07F000C080
:10382000C9F301C0CAF3000E026E0150025C02E14E
:10383000005000080DE201018987640E0501E96F5F
:103840004A0EEA6F000EEB6F42EC08F0B0EC07F0A6
:10385000490E0501E96F020EEA6F6B0EEB6F000E69
:10386000EC6FFAEC07F000C0C9F301C0CAF3000E18
:10387000026E0150025C02E10050000811E2010EEC
:103880000101186F000E196F8997930E0501E96FFA
:10389000450EEA6F000EEB6F42EC08F0B0EC07F05B
:1038A000490E0501E96F020EEA6F740EEB6F000E10
:1038B000EC6FFAEC07F000C0C9F301C0CAF3000EC8
:1038C000026E0150025C02E1005000080FE20101AB
:1038D000186B196B8987F90E0501E96F4B0EEA6FBA
:1038E000000EEB6F42EC08F0B0EC07F0490E05015A
:1038F000E96F020EEA6F970EEB6F000EEC6FFAECB9
:1039000007F000C0C9F301C0CAF3000E026E0150F7
:10391000025C02E1005000081BE2130E0501E96F92
:103920004A0EEA6F000EEB6F42EC08F047C280F5DA
:1039300048C281F59EEC0FF000C0D2F001C0D3F078
:1039400047C280F548C281F554EC0EF0B0EC07F0A8
:10395000490E0501E96F020EEA6FA60EEB6F000E2D
:10396000EC6FFAEC07F000C0C9F301C0CAF3000E17
:10397000026E0150025C02E100500008D8B0CFD0C6
:10398000070E0301C925E96E000ECA21EA6EE9CFD0
:10399000E9FFEACFEAFFEE50310A39E1080EC92506
:1039A0000501E96F000E0301CA210501EA6FAE0EA1
:1039B000EB6F000EEC6FFAEC07F000C0C9F301C02A
:1039C000CAF3000E026E0150025C02E100500008D2
:1039D000D8A08C88080E0301C9250501E96F000EE7
:1039E0000301CA210501EA6F890EEB6F000EEC6F2F
:1039F000FAEC07F000C0C9F301C0CAF3000E026E72
:103A00000150025C02E100500008D8A08C98070E1B
:103A10000301C925E96E000ECA21EA6EE9CFE9FF6C
:103A2000EACFEAFFEE50320A39E1080EC925050156
:103A3000E96F000E0301CA210501EA6F8E0EEB6FDC
:103A4000000EEC6FFAEC07F000C0C9F301C0CAF336
:103A5000000E026E0150025C02E100500008D8A086
:103A60008D88080E0301C9250501E96F000E0301C9
:103A7000CA210501EA6F920EEB6F000EEC6FFAECB3
:103A800007F000C0C9F301C0CAF3000E026E015076
:103A9000025C02E100500008D8A08D98F70E0501E5
:103AA000E96F490EEA6F000EEB6F42EC08F047C277
:103AB000D2F548C2D3F5970E0501D46F4A0ED56FE3
:103AC000000ED66FE9EC0CF00E0E02014725E16EF8
:103AD000000E4821E26E006A8CB8002A300E0026E3
:103AE000E1CFE1FFE2CFE2FF00C0E6FF150E472580
:103AF000E16E000E4821E26E006A8DB8002A300E99
:103B00000026E1CFE1FFE2CFE2FF00C0E6FF47C2BF
:103B100080F548C281F554EC0EF0B0EC07F0490E88
:103B20000501E96F020EEA6F590EEB6F000EEC6FA4
:103B3000FAEC07F000C0C9F301C0CAF3000E026E30
:103B40000150025C02E10050000843E2010189BD1E
:103B500040D0E50E0501E96F4B0EEA6F000EEB6FEA
:103B600042EC08F047C2D2F548C2D3F5A60E0501D3
:103B7000D46F4B0ED56F000ED66FE9EC0CF047C238
:103B800080F548C281F554EC0EF0A60E0501E96FF0
:103B9000480EEA6F000EEB6F42EC08F0690E05016B
:103BA000D26F4D0ED36F000ED46F000E010189B994
:103BB000010E0501D56FD5EC09F0340E0501E96F52
:103BC0004E0EEA6F000EEB6F42EC08F08C8C010198
:103BD000898D490E0501E96F020EEA6F470EEB6F02
:103BE000000EEC6FFAEC07F000C0C9F301C0CAF395
:103BF000000E026E0150025C02E10050000823E258
:103C00006C0E0501E96F4C0EEA6F000EEB6F42EC93
:103C100008F0A70E0201476F010E486F47C2D2F5A8
:103C200048C2D3F5480E0501D46F400ED56F000E83
:103C3000D66FE9EC0CF047C280F548C281F554EC30
:103C40000EF0B0EC07F0490E0501E96F020EEA6FC5
:103C50004C0EEB6F000EEC6FFAEC07F000C0C9F3EE
:103C600001C0CAF3000E026E0150025C02E1005076
:103C7000000870E2BB0E0501E96F4B0EEA6F000E03
:103C8000EB6F42EC08F0FC0E0501D26F4D0ED36FC6
:103C9000000ED46F000E010189B9010E0501D56F28
:103CA000D5EC09F03D0E0B6EE10E0C6E3F0E0D6E65
:103CB0000D2EFED70C2EFCD70B2EFAD700000000DD
:103CC000490E0501E96F020EEA6F79EC07F039EC55
:103CD00008F0490E0501E96F020EEA6F560EEB6F10
:103CE000000EEC6FFAEC07F000C0C9F301C0CAF394
:103CF000000E026E0150025C02E10050000827E253
:103D0000020E0301C95DE16E000ECA59E26EE1CFF9
:103D1000E1FFE2CFE2FFE66A47C280F548C281F5E3
:103D2000520E0501826F020E836F45EC0DF047C203
:103D3000E9F548C2EAF579EC07F039EC08F047C23A
:103D400080F548C281F554EC0EF0B0EC07F00301A9
:103D5000C96BCA6B010189BD26D03A0E0501E96F16
:103D6000440EEA6F000EEB6F42EC08F0380E0501CE
:103D7000D26F4B0ED36F000ED46F000E010189B9C4
:103D8000010E0501D56FD5EC09F0B70E0B6EA10E33
:103D90000C6EC30E0D6E0D2EFED70C2EFCD70B2E07
:103DA000FAD700000000B0EC07F00101164B172B0A
:103DB000800E006E800E1719005C02E116513B0860
:103DC00009E2866B010E0001D46F010ED56F01016F
:103DD000166B176B7A0E0B6EC10E0C6E810E0D6E8C
:103DE0000D2EFED70C2EFCD70B2EFAD700000000AC
:103DF0007AEC0FF05C0E0B6E510E0C6E600E0D6EB9
:103E00000D2EFED70C2EFCD70B2EFAD70000CD0EB0
:103E10000501F06F030EF16F390EF26F000EF36FB4
:103E2000080EF46F7BEC02F0000E011802E1000EA8
:103E3000001805E1010E0101186F000E196F010154
:103E4000000E191902E1010E181970E1000E006E42
:103E50000001C451005C02E1C351000866E2D70EC4
:103E60000501E96F470EEA6F000EEB6F42EC08F0B8
:103E7000300E010118250501F06FBCEC04F0090EAD
:103E80000501F06FBCEC04F07B0E0501E96F4E0EEE
:103E9000EA6F000EEB6F42EC08F0CD0E0501E96F02
:103EA000030EEA6F79EC07F039EC08F0B0EC07F09C
:103EB000CD0E0501F06F030EF16F420EF26F000E92
:103EC000F36F040EF46F7BEC02F0000E011802E1B8
:103ED000000E001804E10101186B196B22D0CD0E01
:103EE0000501D26F030ED36F2FEC0AF00D0EF06FA9
:103EF000E1EC04F03D0E0B6EE10E0C6E3F0E0D6E0C
:103F00000D2EFED70C2EFCD70B2EFAD7000000008A
:103F1000490E0501E96F020EEA6F79EC07F039EC02
:103F200008F0B0EC07F07AEC0FF089D70001000E32
:103F3000B31902E1020EB2191EE1DA0E0501E96FB2
:103F4000490EEA6F000EEB6F42EC08F0B4C0E9F5E1
:103F5000B5C0EAF5360E0501EB6F010EEC6F70ECA3
:103F600005F0360EE96F010EEA6F79EC07F039ECD7
:103F700008F0B0EC07F080B002D001018997010190
:103F8000000E881902E1000E871901E1F8D7E5EF6C
:043F900017F0FFD750
:104EAA0010EE1AF0B40E006E010E016E940EF66E3C
:0E4EBA003F0EF76E000EF86E2EEC0DF012009B
:053F9400333833370053
:053F99004D41483D0010
:053F9E00434D544900F1
:053FA300343731350048
:033FA8004F4B007C
:023FAB00000014
:063FAD004D4350313D00C0
:093FB3004465627567204F4E0061
:053FBC00457869740066
:053FC10048656C700072
:0A3FC60042617474657269653F0082
:033FD0004F4B0054
:083FD300536F6D6D65696C0010
:0A3FDB00537572766579204F6E0071
:093FE5004465627567204F4E002F
:0A3FEE004465627567204F464600E7
:0B3FF800537572766579204F666600F5
:05400300204F6666007D
:04400800204F6E00D7
:05400C00204F66660074
:0F40110044617461204F6E2044656D616E6400E0
:08402000436465204C65640057
:04402800204F6E00B7
:02402C00000092
:02402E00000090
:074030002B43474D533A00FA
:034037004F4B00EC
:02403A003E0046
:01403C000083
:02403D00000081
:03403F004F4B00E4
:0240420000007C
:0240440000007A
:02404600000078
:104048000D0A4364657320646973706F3A0D0A2022
:1040580044617461204F6E2044656D616E64200D6B
:104068000A20537572766579204F6E20286F752067
:104078004F6666290D0A20536F6D6D65696C0D0AD0
:1040880020436465204C65643120306E20286F75AC
:10409800204F6666290D0A2042617474657269654D
:1040A8003F0D0A204465627567204F4E2F4F4646E4
:0340B8000D0A00EE
:1040BB00205241313D45413120646574656374691B
:1040CB006F6E20696E74727573696F6E20284C4425
:1040DB004452292C2020205241323D454132204D63
:1040EB0065737572652054656D7065726174757258
:1040FB006520766961204C4D3335445A203020E0E1
:08410B00313030B0430D0A0011
:1041130020456E74726565733A2042503120737581
:104123007220524437202C20425032207375722063
:10413300524833200D0A20536F7274696573203A15
:1041430020204C4431207375722052443420202C9B
:10415300204C44322020737572205245340D0A00DE
:1041630020536F75726365203A205F3138463837C4
:104173004A35305F47534D325F55415254325F5594
:10418300415254315F574F455F4C4D3335445A5F6D
:10419300323032342D30342E63205F207265762026
:0F41A30032342D30342D323032342E630D0A0079
:1041B2002050726F6A65743A2031384638374A3572
:1041C200305F47534D325F4750535F374E5F554123
:1041D2005254325F55415254315F4C43445F49322D
:1041E200435F4D435032333031375F574F455F3273
:0F41F2003032342D30342E6D637070690D0A0039
:10420100204469726563746F7279203A433A5C5F46
:104211004D696B726F435C5F4D657350726F6A6578
:1042210074735F4D696B726F435C5F313846383729
:104231004A35305F47534D325F515545434B5445E5
:0D4241004C5F4D39355F323032340D0A00CC
:10424E0020526571756574652044617465205469EA
:10425E006D652061752073657276657572204E549A
:10426E0050204364653D41542B514E54503D2231F4
:10427E0033302E37392E31342E313737222C31321E
:05428E0033290D0A00B8
:10429300204D696B726F4520436C69636B657232A5
:1042A3002031384634374A3530202B2047534D20B0
:1042B3005175656374656C204D393520636C696392
:1042C3006B20737572204D6963726F42757323316E
:0442D300200D0A00B0
:1042D70020456E7265676973747265204E756D65EA
:1042E700726F2074656C204A6F656C6C65202C6555
:1042F7006E20706F736974696F6E2053494D203259
:10430700202841542B435042573D322C2E2E290D45
:024317000A009A
:1043190020456E7265676973747265204E756D65A7
:10432900726F2074656C205061756C202C656E204D
:10433900706F736974696F6E2053494D203120285D
:1043490041542B435042573D312C2E2E290D0A0042
:10435900205175657279207468652073746174756C
:1043690073206F662053494D2063617264206C6F1E
:10437900636B2C20302D756E6C6F636B2028415454
:0F4389002B434C434B3D225343222C320D0A0051
:1043980020436F6D70696C6174696F6E2053414E74
:1043A8005320627573204932432C20646F6E63205A
:1043B80073616E73204C43442C206E69204D43502A
:0843C80032333031370D0A00D9
:1043D000204C69737420616C6C20554E52454144E9
:1043E000206D73672066726F6D20696E626F782032
:1043F0002841542B434D474C3D52454320554E5286
:07440000454144290D0A00AB
:104407002055415254312031393230302C382C4E1E
:104417002C31203C2D3E207465726D696E616C20D5
:1044270053414E5320475053206163746976E92006
:034437000D0A006B
:10443A0045666661636520746F7573206C657320C9
:10444A00534D53207265E77573202841542B514D03
:10445A004744413D2244454C20494E424F58222967
:03446A000D0A0038
:10446D0045666661636520746F7573206C65732096
:10447D00534D53207265E77573202841542B514DD0
:10448D004744413D2244454C20494E424F58222934
:03449D000D0A0005
:1044A00020636C69676E6F7465204C443120656EC3
:1044B000207065726D616E656E6365202C72657328
:1044C0006574206E6563657373616972652E2E0D68
:0244D0000A00E0
:1044D20020557361676520646520534C4545502023
:1044E2006D6F646520302065742032202C766961FE
:1044F20020436465206C69676E6520445452200D28
:024502000A00AD
:1045040020554152543220393630302C382C4E2C20
:104514003120706F75722047534D322D436C69639F
:104524006B205155454354454C204D3935200D0AD7
:014534000086
:10453500205265667573E965200D0A205042206496
:104545006520666F726D617420636465203A204D45
:0F4555004350313D30303030303030300D0A00BF
:104564002052656164206D657373616765204E4FE9
:104574004E204C5553202841542B434D474C3D224B
:0F45840052454320554E5245414422290D0A000D
:10459300204445425547206D6F6465204F4E200DE2
:1045A3000A20417474656E74652063646520636CCE
:0F45B3006176696572202D3E2047534D0D0A0039
:1045C20041542B435042573D322C222B3333363148
:1045D20034313333383337222C3134352C224A6F7D
:0D45E200656C6C65222C31322C31320D00DD
:1045EF00222B3333363231333334373135220022F5
:1045FF002B333336313431333338333722004E6F68
:0D460F007420617574686F72697A656400CB
:10461C0041542B435042573D312C222B33333632ED
:10462C0031333334373135222C3134352C2250612F
:0B463C00756C222C31322C31320D0045
:10464700200D0A20436F6E737469747574696F6EF9
:104657002062617365206427756E20534D5320E0F7
:0B46670020656E766F7965720D0A0009
:104672002052656E766F6920534D532073757220F8
:104682007465726D696E616C202841542B434E4DE6
:0A469200493D322C3129200D0A00A9
:10469C0020466F726365204E6574776F726B207263
:1046AC006567697374726174696F6E202841542B4D
:0A46BC00435245473D30290D0A0026
:1046C6002053656E64204D73672074797065206190
:1046D600732074657874206D6F6465202841542BAF
:0A46E600434D47463D31290D0A00FF
:1046F0002052654C65637475726520646520646141
:104700007465206574206865757265202841542B96
:0947100043434C4B3F290D0A0004
:1047190020466F726D6174206465205265706F6EFA
:10472900736520766961206C6962656C6CE9202883
:0847390041545631290D0A001C
:10474100204E6576657220676F20696E20534C4557
:104751004550206D6F64652841542B5153434C4B98
:064761003D30290D0A00A5
:104767004E6576657220476F20696E20534C45452C
:1047770050206D6F64652841542B5153434C4B3D7A
:064787003029200D0A009C
:10478D002044656C6C20416C6C20534D53202841A6
:10479D00542B514D4744413D2244454C20414C4CF6
:0547AD0022290D0A00A5
:1047B2002053656C65637420534D202841542B436C
:1047C200504D533D22534D222C22534D222C225325
:0547D2004D220D0A005C
:1047D700204D6F6465204465627567203C457869A4
:1047E700743E20706F757220656E20736F727469E6
:0447F70072203D00EF
:1047FB002031657265204C65637475726520414488
:10480B0043205241312065742041444320524132B0
:04481B00203A20001F
:10481F0020517565727920736572766963652063BF
:10482F00656E7465722E2841542B435343413F29C3
:03483F000D0A005F
:1048420020204D6F6E69746F7220506F77657220F1
:10485200537570706C79282041542B4342432920B0
:034862000D0A003C
:1048650020494D45492053657269616C206E756D0F
:10487500626572202841542B4347534E29200D0A67
:014885000032
:1048860020506F776572204F4E206D6F64756C6592
:104896002047534D322D636C69636B200D0A20004F
:1048A600476F20696E20534C454550206D6F6465F7
:1048B6002841542B5153434C4B3D3229200D0A00BD
:1048C60041542B43434C4B3D2231352F30392F3247
:1048D600392C31363A34353A30302B3034220D000B
:1048E60020536F6674776172652056657273696FBF
:0F48F6006E202841542B43474D5229200D0A00B4
:10490500205265667573E96520636172204D4350D9
:0F491500323330313720616273656E740D0A00E2
:104924000D0A496E697420657420316572204465EE
:0F4934006D6172726167652047534D320D0A0045
:10494300204574617420696E69742047534D202893
:0F49530041542B51494E4953544154290D0A00E8
:1049620020313932303020426175642072617465C1
:0F497200204E65676F636520424144200D0A00A7
:10498100200D0A20436F6E74656E75206475205387
:0F4991004D5320E020656E766F7965720D0A0038
:1049A000436865636B202050494E20636F6465281F
:0D49B00041542B4350494E3F29200D0A0071
:1049BD0041542B514E54503D223133302E37392E28
:0D49CD0031342E313737222C3132330D00BA
:1049DA00204465626F7264656D656E7420627566E7
:0D49EA00666572205541525432200D0A00BE
:1049F700205265746F75722064276F726472652028
:0C4A0700636465204C656473200D0A0098
:104A13000D0A456E766F6920446174617320646585
:0B4A23006D616E64E96573200D0A00F0
:104A2E002046756C6C20696E69742047534D206565
:0B4A3E006E203139207061730D0A00FA
:104A4900205072657420706F757220656E766F697B
:0B4A5900204D7367205478200D0A00E8
:104A6400204469616C6F67756520534D53207265EE
:0A4A74007461626C6974200D0A0081
:104A7E00204572726575722073757220656E766F41
:094A8E006920534D53200D0A006C
:104A97000D0A5265746F7572204C6564313D202094
:084AA7004C6564323D200D0056
:104AAF0041542B43504D533D22534D222C22534DF5
:084ABF00222C22534D220D00B0
:104AC70020536176652070726F66696C6520284196
:074AD700542657290D0A00C7
:104ADE002041726D65205258204954205541525440
:074AEE0031202E2E0D0A00FD
:104AF5002041726D65205258204954205541525429
:074B050032202E2E0D0A00E4
:104B0C000D0A47534D322050494331384638374A05
:064B1C0035303A0D0A00DD
:104B220041542B434D474C3D2252454320554E5252
:064B3200454144220D0084
:104B380041542B514D4744413D2244454C20494E58
:064B4800424F58220D004F
:104B4E0041542B434D474C3D2252454320554E5226
:064B5E00454144220D0058
:104B64002053544F50206469616C6F6775652053FE
:064B74004D53200D0A0064
:104B7A000D0A2050686F6E6573204E756D626572FE
:064B8A0073203A0D0A0041
:104B900041542B514D4744413D2244454C20494E00
:064BA000424F58220D00F7
:104BA6000D0A4F4B206D6F6465206D696D696E75DA
:054BB6006D20780D00E8
:104BBB005265E775204364652042617474657269C0
:054BCB00653F0D0A002A
:104BD000204E65676F636520626175642072617441
:054BE00065200D0A0034
:104BE500204D69736520656E20736F6D6D65696C09
:044BF500200D0A0085
:104BF9002053544F50206D6F64652064656275675A
:044C0900200D0A0070
:104C0D00204D414A206461746520657420486575A6
:044C1D00726520009C
:104C210041542B434D474C3D2244454C20414C4C73
:034C3100220D0051
:104C340020436F6D706F7365204D7367206C656ED4
:034C44003D200010
:104C470020506173206465204D4350323330313733
:034C570021200019
:104C5A00205068617365206427696E697420656EE7
:024C6A00200028
:104C6C002048656C702064656D616E64E965200D8B
:024C7C000A002C
:104C7E00204E65676F636520726575737369200DCD
:024C8E000A001A
:104C900020436F6D706F7365204E756D65726F2068
:014CA0000013
:104CA10052657665696C2047534D32202F4454522A
:014CB1000002
:104CB200202E2E20706173205072657420210D0AFF
:014CC20000F1
:104CC3003B2E2E2E2066696C746572696E67200018
:104CD30020456E766F6920534D53204F4B203A0089
:104CE30041542B434C434B3D225343222C320D0062
:0F4CF30020486172647761726520203A0D0A00D3
:0E4D020020416C61726D2E54656D703D200075
:0E4D100020496E747275732E4541313D2000AE
:0D4D1E0041542B434E4D493D322C310D00C8
:0D4D2B002041444320496E6974200D0A00A8
:0D4D380041542B51494E49535441540D0034
:0C4D4500436465204D435031203A2000AB
:0C4D510041542B5153434C4B3D300D009E
:0C4D5D0041542B5153434C4B3D300D0092
:0C4D690041542B5153434C4B3D320D0084
:0B4D750041542B435245473D300D00D8
:0B4D800041542B434D47463D310D00D0
:0A4D8B000D0A20456E642E0D0A008B
:0A4D950041542B43434C4B3F0D00EB
:0A4D9F0041542B435343413F0D00E4
:0A4DA9002E2E2E20537465703A0080
:0A4DB30041542B43474D520D0A00F6
:0A4DBD0041542B4350494E3F0D00B6
:094DC70020464F5343203D20001B
:094DD0003B4469616C6F673D0012
:094DD90041542B434D47533D00AA
:094DE20041542B4347534E0D00D0
:094DEB003B54656D70463D20004B
:084DF40041542B4342430D0022
:084DFC0041542B4342430D001A
:084E040020425032203D200045
:084E0C002054656D703D20008B
:084E140020425031203D200036
:084E1C00204C4431203D200030
:084E24003B20535441543D00B2
:084E2C00207061732F31390081
:084E34004454523D310D0A0007
:084E3C00204C4432203D20000F
:074E44003B204250323D000B
:074E4B003B204541323D0010
:074E52002E2E424144210015
:074E59003B204C44313D00F9
:074E60003B20534F4D3D00C4
:074E67003B204454523D00C2
:074E6E003B204C44323D00E3
:064E75002E2E204F4B0021
:064E7B00204364653D00C8
:064E81004541313D200017
:064E8700415426570D0006
:064E8D006465672043008C
:064E93003B4250313D00DE
:064E9900204541313D00FF
:064E9F00415456310D00E4
:044EA50041540D0067
:020000040001F9
:06FFF800ACF7C5FFF8FFA5
:00000001FF
